:1000000024C048C047C046C045C044C043C042C0E9
:1000100041C040C03FC001C83DC03CC03BC03AC029
:1000200039C038C037C036C035C034C033C032C024
:1000300031C030C02FC02EC02DC02CC001020480A2
:100040004020100804020108FE0311241FBECFEF58
:10005000D2E0DEBFCDBF11E0A0E0B1E0E0EAFAE11E
:1000600002C005900D92A432B107D9F721E0A4E2B5
:10007000B1E001C01D92A038B207E1F710E0C5E27F
:10008000D0E003C02197FE016FDCC432D107D1F765
:10009000B7D904CDB5CF98E09A95F1F708950895B2
:1000A000B7E0A0ED002409D032F40A94E1F71197EB
:1000B000C9F7289408C0A89406C0A894CC9901C098
:1000C0002894000008950895D698D498DE98DC9876
:1000D00088279927CE9B0895CC9B089581E00895A9
:1000E00081E00895D49AD7DFD698D5DFD498D3DFAE
:1000F000CC9BD6DFD69ACFDF21D0089581E008953A
:100100008F93F1E0E4EF8F918F93CC9BC9DFD69A68
:10011000C2DF14D0882321F407D0319709F0F3CF40
:1001200099270F9008950895D49AD69AB4DFD49859
:10013000B2DFCC9BB5DFD698AEDF08950894881F58
:1001400001C0880FB9F0D49A00000000000018F434
:100150000000D69802C0D69A00C09DDFD498A8941B
:10016000000000000000CC9B9BDF12F4882712C027
:1001700092DFE7CFD49A00000000D6988CDF992751
:100180008827D498A8940000CC9B8ADF7AF3CE9B72
:1001900081E081DF00000000D49A089581E0089595
:1001A00071E0D49AD69800000000000074DFD49863
:1001B00072DFA894000000000000CC9B71DFB2F059
:1001C0008894CE990894771F60F7D49A803011F004
:1001D000D69801C0D69A0000000000005CDFD498D9
:1001E000A89400000000CC9B5BDF55DF00000000FE
:1001F000D49A872F9927089580E2089580916E01FF
:1002000090916F0190936D0180936C0180916E01CC
:1002100090916F01019690936F0180936E01809190
:100220006E0190916F018F3F910529F024F010929B
:100230006F0110926E0180916E0190916F0160913B
:1002400071011EDC80916C0190916D016FEF18CCF3
:10025000CF93DF93C0E0D0E0CE010ADC8F3F39F0CE
:10026000D0936F01C0936E018093710104C02196F9
:10027000CF3FD10589F790917101809118019817AE
:1002800010F010927101DF91CF91089510927501D5
:10029000809171018F5F809371019091180189178E
:1002A00010F010927101AACF109275018091710126
:1002B000815080937101A2CF1F93CF93DF931F9240
:1002C000CDB7DEB7182F8CEE1BDF812F37DF8DEE19
:1002D00009DF81E065DF898327DF89810F90DF9166
:1002E000CF911F91089580E0E7DF90E0813891057C
:1002F00014F080E890E00895CF93C82F63D78C2F37
:10030000CF9160C7CF93DF93EC01892B11F460E0AC
:1003100005C0CF3F83E0D80718F061E083E0ADD798
:100320008091CA008F7E8093CA008091CA0080624B
:100330008093CA00D093C300C093C200D0937301CE
:10034000C0937201DF91CF910895AF92BF92CF9287
:10035000DF92EF92FF920F931F93CF93DF936B0186
:10036000EC0197FF02C0C0E0D0E061E08AE085D7F1
:1003700000E010E05E0185E0A81AB1080D2C000C29
:10038000EE08FF080A151B0544F40B5F1F4FC80158
:10039000B9DFC701B601BED6F5CFCE01DF91CF914F
:1003A0001F910F91FF90EF90DF90CF90BF90AF9093
:1003B000A9CFCF92DF92EF92FF920F931F93CF932B
:1003C000DF93EC018B016B01770FEE08FF081C1621
:1003D0001D0644F4C01BD10BCE0194DFC701B6014A
:1003E00099D6F5CF60E08AE0DF91CF911F910F9110
:1003F000FF90EF90DF90CF9040C7CF93DF93D82F3F
:1004000062E070E08091720190917301D2DF60E050
:100410008AE033D768EC70E080E090E07BD682E041
:1004200090E070DFC0E0CD1791F061E08AE025D761
:1004300069EE70E080E090E06DD660E08AE01DD764
:100440006CE271E080E090E065D6CF5FECCFDF91A9
:10045000CF91089583E0D1CF85E0CFDF1092710175
:10046000CDDEFFCF81E048DF20917101211110C066
:10047000813C910534F4809175018F5F8093750103
:1004800002C010927501809175018A30A0F0E4DFFE
:10049000823D910534F4809175018F5F80937501E1
:1004A00002C010927501809175018A3020F010927F
:1004B0007001D0DFF9CE089584E09FDF10927101C2
:1004C0009DDEFFCF10DF20911001309111018217C6
:1004D00093070CF0F1DF0895CF92DF92EF92FF9235
:1004E00081E08093700180917001813081F5BADFE5
:1004F000E9DF62E070E080E090E060D76B017C01B2
:1005000062E070E080E090E059D724E0C20ED11C98
:10051000C601861B970BF6DE66E470E080E090E093
:100520004DD76B017C0162E370E080E090E046D73C
:10053000C60ED71EE81EF91E64E170E080E090E070
:100540003DD76C0D7D1D8E1D9F1DE4D5CCCFFF903A
:10055000EF90DF90CF900895CF92DF92EF92FF92CD
:100560000F931F93CF93DF93E82FF0E0EE0FFF1F61
:10057000E75EFE4FC081D18180E090E0C3DE61E0A4
:100580008AE07BD6CF3F2FEFD20711F4A5DF22C040
:10059000C734D105FCF0BE010D2E000C880B990B61
:1005A00032D86B017C018B019C0140E050E060E798
:1005B00072E484E291E078D3C0926001D09261014C
:1005C000E0926201F092630184E291E0E8D381E07D
:1005D0008093740181E090DE8930914074F4C330DF
:1005E00082E0D80754F060DEDF91CF911F910F9128
:1005F000FF90EF90DF90CF902DCF68E070E0CE01BC
:10060000DF91CF911F910F91FF90EF90DF90CF90EE
:100610009CCECF93DF9380E08CD6EC0181E089D62D
:10062000C130D105C1F4892B91F584E08093180184
:1006300088E090E090931C0180931B0183E191E09E
:100640009093200180931F01809171018430F8F014
:10065000109271011CC0CD2BD1F48130910549F469
:1006600088E090E090931C0180931B0186ED92E05E
:100670000AC0892B61F488E090E090931C0180937C
:100680001B018AEA93E09093220180932101DF917C
:10069000CF910895CF93DF9380E091D561E087E01B
:1006A000A6D560E088E0A3D582E026DEEC01D0DDAF
:1006B000CB3FD10514F0EADD06C08091160181110F
:1006C00002C01092710161E083E091D561E08AE09F
:1006D0008ED561E088E08BD562E080E088D562E06D
:1006E00081E085D560E081E082D561E088E0C5D514
:1006F00060E08AE0C2D560E083E0BFD58ADF7EDDBE
:100700008091C900887F81608093C9008091C90071
:100710008F7E8093C9008091C90088608093C90052
:100720008091CA0082608093CA008091CA00816073
:100730008093CA00C9DC811101C0BEDED4DDBC01DA
:10074000990F880B990B5FD76093640170936501D3
:10075000809366019093670180911201909113013B
:10076000A0911401B09115018093680190936901E3
:10077000A0936A01B0936B0161E084E291E0DF91A4
:10078000CF9151C38091710190911701891719F090
:1007900080931701E1DE80917401813019F592DEBA
:1007A00061DE69E170E080E090E0B4D49CDDBC01E2
:1007B000990F880B990B27D760936401709365019B
:1007C000809366019093670184E291E055D0609137
:1007D0006001709161018091620190916301E5D6A1
:1007E000CB0190CD6FDE69E170E080E090E092D4C3
:1007F00039DE69EA71E080E090E08CC4AF92BF928C
:10080000CF92DF92EF92FF920F931F93A090080177
:10081000B0900901C0900A01D0900B01E0900C014A
:10082000F0900D0100910E0110910F011F921F9287
:10083000809107018F93809106018F93809105012C
:100840008F93809104018F9328E631E040E651E0D8
:1008500064E671E084E291E0A0D30F900F900F90D6
:100860000F900F900F901F910F91FF90EF90DF90DE
:10087000CF90BF90AF9008952F923F924F925F928A
:100880006F927F928F929F92AF92BF92CF92DF92A0
:10089000EF92FF920F931F93CF93DF93CDB7DEB705
:1008A00060970FB6F894DEBF0FBECDBFDC01DA96BD
:1008B000BC91B983B11102C0198218C1988B8F877E
:1008C000F6D36E837F8388879987EF85F88982A125
:1008D00093A1A4A1B5A14E815F8168857985481B4C
:1008E000590B6A0B7B0B86A597A5A0A9B1A9481740
:1008F00059076A077B0700F3248D358DD9018D9147
:100900009D910D90BC91A02D8A839B83AC83BD8368
:1009100000A0F1A1E02D9C01AD0160817181828177
:10092000938172D54B015C01EF85F88922A533A52F
:1009300044A555A56A817B818C819D8165D56B011C
:100940007C01AF85B88950962D913D914D915C9178
:100950005397C501B4010BD7EF85F88926A137A1BC
:1009600040A551A552D52B013C01AF85B88996967B
:100970006D937D938D939C939997DB96BC91BA87E9
:10098000B11116C0EF85F8892485358546855785D0
:10099000C701B601ECD69B01AC01C301B20134D54D
:1009A000AF85B88996966D937D938D939C93999717
:1009B000EF85F88946A057A060A471A416A907A9DD
:1009C00030AC21AC212F302F432D522DC301B20169
:1009D000CAD618162CF4812F902FA32DB22D17C034
:1009E000AF85B889D2968D919D910D90BC91A02D27
:1009F0008B879C87AD87BE879C01AD01C301B20187
:100A000068D587FF0AC08B859C85AD85BE85EF853F
:100A1000F88986A397A3A0A7B1A7FA85FF2371F051
:100A2000AF85B8891C962D913D914D915C911F9792
:100A3000C501B4019CD64B015C0103C0812C912CF3
:100A40005401EF85F8892489358946895789C7017A
:100A5000B6018DD69B01AC01AF85B88996966D9194
:100A60007D918D919C919997CFD49B01AC01C5014B
:100A7000B401CBD46B017C01212F302F432D522D9B
:100A800072D618169CF0EF85F88912A903A934A82C
:100A900025A8212F302F432D522DB601C70119D57E
:100AA00087FD04C01C2D0D2D3E2C2F2CAF85B88941
:100AB0005E96ED91FC915F97812F902FA32DB22D23
:100AC00080839183A283B3838A819B81AC81BD8122
:100AD000EF85F88982A793A7A4A7B5A78E819F81E8
:100AE000A885B98582A393A3A4A3B5A389816096A1
:100AF0000FB6F894DEBF0FBECDBFDF91CF911F912F
:100B00000F91FF90EF90DF90CF90BF90AF909F90AC
:100B10008F907F906F905F904F903F902F900895AF
:100B20002F923F924F925F926F927F928F929F92FD
:100B3000AF92BF92CF92DF92EF92FF920F931F93EB
:100B4000CF93DF9300D000D0CDB7DEB71C0149832F
:100B50005A836B837C832801390120E030E0A901AE
:100B600069817A818B819C81B4D487FD86C020E025
:100B700030E0A901C301B201ACD487FD7EC020E002
:100B800030E0A901C701B601A4D487FD76C0D10128
:100B90005B96BC92AE925A9781E0AA94AB2809F07A
:100BA00080E0F10183AF89819A81AB81BC81808330
:100BB0009183A283B3834482558266827782C08602
:100BC000D186E286F38666A577A580A991A919D575
:100BD00020E030E04AE754E480D44B015C01898195
:100BE0009A81AB81BC81F10184879587A687B787FD
:100BF000A5019401C301B201BAD52B013C01D10179
:100C000050966D937D938D939C935397A50194017A
:100C1000C701B60162D46B017C01F101648B758B55
:100C2000868B978B808D918D019739F529813A813B
:100C30004B815C8160E070E0CB01E6D3D1011C9672
:100C40006D937D938D939C931F97A301920160E018
:100C500070E0CB01D9D3F101608B718B828B938BC8
:100C6000A701960160E070E0CB01CED3D10154968C
:100C70006D937D938D939C9357970F900F900F904A
:100C80000F90DF91CF911F910F91FF90EF90DF9028
:100C9000CF90BF90AF909F908F907F906F905F901C
:100CA0004F903F902F9008952F923F924F925F92D6
:100CB0006F927F928F929F92AF92BF92CF92DF926C
:100CC000EF92FF920F931F93CF93DF93EC016A0192
:100CD0007B0148015901A9019801C701B60143D51B
:100CE00087FF4AC0CAAADBAAECAAFDAA8EAA9FAABD
:100CF000A8AEB9AE8AAD882309F43EC02E8C3F8CD5
:100D0000F1014080518062807380A5019401C3018C
:100D1000B20129D5181634F4F10180829182A282A1
:100D2000B3820CC0A7019601C301B201D2D387FFE1
:100D300005C0F101C082D182E282F3828EA09FA021
:100D4000A8A4B9A4CEA8DFA8E8ACF9ACA701960185
:100D5000C501B40108D518165CF0CAA8DBA8ECA838
:100D6000FDA8A7019601C501B401B3D387FF04C054
:100D7000CEA2DFA2E8A6F9A6DF91CF911F910F9135
:100D8000FF90EF90DF90CF90BF90AF909F908F90AB
:100D90007F906F905F904F903F902F9008958F922B
:100DA0009F92AF92BF92CF92DF92EF92FF92CF933A
:100DB000DF93EC01EE8DFF8DC080D180E280F38067
:100DC000CEA2DFA2E8A6F9A6EC8DFD8D80819181EF
:100DD000A281B3818AA79BA7ACA7BDA78EA89FA815
:100DE000A8ACB9ACA5019401C701B601BCD41816D2
:100DF0005CF08AA89BA8ACA8BDA8A5019401C70176
:100E0000B60167D387FF04C08EA29FA2A8A6B9A689
:100E1000DF91CF91FF90EF90DF90CF90BF90AF9098
:100E20009F908F9008951F93CF93DF93EC0111E073
:100E3000613011F010E005C08AAD811102C0CE0111
:100E4000AEDF1AAFDF91CF911F9108950F931F93DB
:100E5000CF93DF93EC018B018AAD882349F1888D14
:100E6000998D6817790721F12C853D854E855F8521
:100E700060E070E0CB01C8D26C877D878E879F874A
:100E8000288939894A895B8960E070E0CB01BCD24E
:100E9000688B798B8A8B9B8B2C893D894E895F89E6
:100EA00060E070E0CB01B0D26C8B7D8B8E8B9F8B22
:100EB000198F088FDF91CF911F910F9108954F9255
:100EC0005F926F927F928F929F92AF92BF92CF92DA
:100ED000DF92EF92FF920F931F93CF93DF9300D097
:100EE00000D0CDB7DEB74C0127013801A982BA8204
:100EF000CB82DC82FC01578F468F758F648F31A3C4
:100F000020A312AE12AA13AA14AA15AA80E090E098
:100F1000AFE7B3E486AB97ABA0AFB1AF84E690E0A8
:100F2000A0E0B0E086A797A7A0ABB1AB6D8D7E8D9A
:100F3000C4018CDFAB8CBC8CCF88D88CE98CFA8C4C
:100F400009811A812B813C81B301A201C401E8DD32
:100F5000AED0F40106A517A520A931A9DC01CB016B
:100F6000801B910BA20BB30B82A393A3A4A3B5A3E5
:100F70000F900F900F900F90DF91CF911F910F91D5
:100F8000FF90EF90DF90CF90BF90AF909F908F90A9
:100F90007F906F905F904F9008958F929F92AF9245
:100FA000BF92CF92DF92EF92FF920F931F93CF9356
:100FB000DF93CDB7DEB7EF85F889A989BA899B8819
:100FC0008C888F929F921F92992493949F92BF93A3
:100FD000AF93FF93EF9373DF0FB6F894DEBF0FBEAE
:100FE000CDBFDF91CF911F910F91FF90EF90DF90D8
:100FF000CF90BF90AF909F908F9008958EB5887FCF
:101000008EBD8FB58C7F81608FBD8EB5877E8EBD86
:101010008EB5887F83608EBD08951F920F920FB6A4
:101020000F9211242F933F938F939F93AF93BF936E
:101030008091770190917801A0917901B0917A0126
:101040003091760126E0230F2D3730F029E8230F69
:101050000396A11DB11D03C00296A11DB11D2093D1
:1010600076018093770190937801A0937901B093F2
:101070007A0180917B0190917C01A0917D01B091DA
:101080007E010196A11DB11D80937B0190937C018F
:10109000A0937D01B0937E01BF91AF919F918F91FD
:1010A0003F912F910F900FBE0F901F9018952FB763
:1010B000F894609177017091780180917901909115
:1010C0007A012FBF08953FB7F89480917B019091EA
:1010D0007C01A0917D01B0917E0122B708B600FE8F
:1010E00005C02F3F19F00196A11DB11D3FBFBA2FBA
:1010F000A92F982F8827820F911DA11DB11DBC011A
:10110000CD0143E0660F771F881F991F4A95D1F7DD
:1011100008950895CF92DF92EF92FF92CF93DF93DD
:101120006B017C01D0DFEB01C114D104E104F104B7
:1011300079F0EFDFC8DF6C1B7D0B683E7340A0F3D6
:1011400081E0C81AD108E108F108C851DC4FF2CF9C
:10115000DF91CF91FF90EF90DF90CF90089578943A
:1011600080B7836080BF83B7877F83BF83B7887F63
:10117000836083BF89B7816089BF40DFE9ECF0E01D
:101180008081887F808380E18093670084EA8093F8
:1011900068008CEF80936600AAECB0E08C918C7FA5
:1011A00081608C938081877E80838081887F83604B
:1011B000808385B1887F866085B92F9A0895809352
:1011C0007F01089586FD8F7398B120917F0122954C
:1011D000220F207E9F71922B98B999B1907C892B18
:1011E00089B92E9A2E99FECF86B197B10895CF93E3
:1011F000DF9386FF04C08F739BE0981B892FE82F35
:10120000F0E0E45CFF4F94918B3049F0833038F08C
:10121000EBE3F0E0AAE3B0E0C3E6D0E006C0E8E329
:10122000F0E0A7E3B0E0C2E6D0E0892F80952FB7C9
:1012300061110BC0F8949C9198239C939081982302
:10124000908398818923888314C0623059F4F8947C
:101250003C9183238C938081892B8083E881E92BC7
:10126000E88307C0F894388183238883EC91E92BC5
:10127000EC932FBFDF91CF910895CF93DF9386FF3B
:1012800004C08F739BE0981B892FE82FF0E0E45C8B
:10129000FF4FE4918B3051F1833038F091E086308C
:1012A00029F480B78F7380BF26C092E0853021F487
:1012B00080B78F7C80BF18C0843019F48FB58F73CE
:1012C00004C0873021F48FB58F7C8FBD0DC0823074
:1012D00021F48091CA008F7305C0833029F4809176
:1012E000CA008F7C8093CA00913029F0C8E3D0E017
:1012F000A2E6B0E004C0CBE3D0E0A3E6B0E08E2FDE
:10130000809561110AC02FB7F8949881982398832B
:101310009C9189238C932FBF09C09FB7F894288193
:10132000E22BE8832C9182238C939FBFDF91CF9196
:10133000089587FF04C08F779BE0981B892FE82FC3
:10134000F0E0E45CFF4FE4918B3051F1833038F0F2
:1013500091E0863029F480B78F7380BF24C092E07B
:10136000853021F480B78F7C80BF18C0843019F499
:101370008FB58F7304C0873021F48FB58F7C8FBDFC
:101380000DC0823021F48091CA008F7305C0833074
:1013900029F48091CA008F7C8093CA00913019F0A3
:1013A000A6E3B0E002C0A9E3B0E08C91E82381E0BD
:1013B00090E019F480E090E008950895CF93DF93D2
:1013C00000D000D0CDB7DEB761157105810591055C
:1013D00069F09B01AC0169833A834B835C833BD307
:1013E00029813A814B815C812DD203C060E070E09D
:1013F000CB010F900F900F900F90DF91CF91089538
:10140000AEDE48D9BFD9FECF5058BB27AA270ED091
:1014100070C161D130F066D120F031F49F3F11F4FA
:101420001EF456C10EF4E095E7FB4CC1E92F72D1D2
:1014300080F3BA17620773078407950718F071F4F1
:101440009EF58AC10EF4E0950B2EBA2FA02D0B014C
:10145000B90190010C01CA01A0011124FF27591BF9
:1014600099F0593F50F4503E68F11A16F040A22FFF
:10147000232F342F4427585FF3CF46953795279570
:10148000A795F0405395C9F77EF41F16BA0B620B6F
:10149000730B840BBAF09150A1F0FF0FBB1F661FB6
:1014A000771F881FC2F70EC0BA0F621F731F841FF9
:1014B00048F4879577956795B795F7959E3F08F01F
:1014C000B3CF9395880F08F09927EE0F97958795DE
:1014D0000895D4D008F481E008950CD00AC102D157
:1014E00040F0F9D030F021F45F3F19F0EBC051111A
:1014F00034C1EEC00FD198F39923C9F35523B1F34A
:10150000951B550BBB27AA2762177307840738F072
:101510009F5F5F4F220F331F441FAA1FA9F333D0D1
:101520000E2E3AF0E0E830D091505040E695001C85
:10153000CAF729D0FE2F27D0660F771F881FBB1F41
:10154000261737074807AB07B0E809F0BB0B802D1B
:10155000BF01FF2793585F4F2AF09E3F510568F067
:10156000B1C0FBC05F3FECF3983EDCF38695779506
:101570006795B795F7959F5FC9F7880F911D969569
:10158000879597F90895E1E0660F771F881FBB1FC5
:10159000621773078407BA0720F0621B730B840B72
:1015A000BA0BEE1F88F7E0950895BCD088F09F57DE
:1015B00090F0B92F9927B751A0F0D1F0660F771F9F
:1015C000881F991F1AF0BA95C9F712C0B13081F07F
:1015D000C3D0B1E00895C0C0672F782F8827B85FC7
:1015E00039F0B93FCCF3869577956795B395D9F7E0
:1015F0003EF490958095709561957F4F8F4F9F4FEA
:101600000895E89409C097FB3EF4909580957095F5
:1016100061957F4F8F4F9F4F9923A9F0F92F96E93E
:10162000BB279395F695879577956795B795F111B3
:10163000F8CFFAF4BB0F11F460FF1BC06F5F7F4F50
:101640008F4F9F4F16C0882311F096E911C0772362
:1016500021F09EE8872F762F05C0662371F096E86B
:10166000862F70E060E02AF09A95660F771F881F3A
:10167000DAF7880F9695879597F90895990F0008DE
:10168000550FAA0BE0E8FEEF16161706E807F90754
:10169000C0F012161306E407F50798F0621B730BEF
:1016A000840B950B39F40A2661F0232B242B252B70
:1016B00021F408950A2609F4A140A6958FEF811D13
:1016C000811D089597F99F6780E870E060E00895B4
:1016D0009FEF80EC089500240A941616170618064A
:1016E0000906089500240A94121613061406050626
:1016F0000895092E0394000C11F4882352F0BB0FB7
:1017000040F4BF2B11F460FF04C06F5F7F4F8F4F19
:101710009F4F089557FD9058440F551F59F05F3F54
:1017200071F04795880F97FB991F61F09F3F79F003
:1017300087950895121613061406551FF2CF469585
:10174000F1DF08C0161617061806991FF1CF869507
:101750007105610508940895E894BB2766277727EB
:10176000CB0197F908958ADF08F48FEF08950AD026
:10177000C0CFB1DF28F0B6DF18F0952309F0A2CF73
:10178000A7CFEBCFC7DFA8F39923D9F35523C9F32C
:10179000950F50E0551FAA27EE27FF27BB270024EF
:1017A0000894679520F4E20FF31FB41F0A1E220F5E
:1017B000331F441FAA1F6695A9F7779530F4F30FDE
:1017C000B41F0A1E121E08F46395330F441FAA1F8C
:1017D000221F769599F7879520F4B40F0A1E121EE2
:1017E000631F440FAA1F221F331F8695A9F7862F58
:1017F000712D602D11249F5750408AF0E1F088230D
:101800004AF0EE0FFF1FBB1F661F771F881F915006
:101810005040A9F79E3F510570F054CF9ECF5F3FD7
:10182000ECF3983EDCF3869577956795B795F79539
:10183000E7959F5FC1F7FE2B880F911D96958795C1
:1018400097F90895052E97FB16F400940FD057FDD5
:1018500005D068D007FC02D046F408C050954095EA
:10186000309521953F4F4F4F5F4F0895909580954C
:10187000709561957F4F8F4F9F4F08956894001327
:10188000E894A0E0B0E0E6E4FCE01DC0EFEFE7F98B
:1018900059016A015E23550FEE08FE2C87019B015A
:1018A000AC019E23990F660B762FCB0163D0CDB789
:1018B000DEB7EAE024C02F923F924F925F926F9280
:1018C0007F928F929F92AF92BF92CF92DF92EF92D0
:1018D000FF920F931F93CF93DF93CDB7DEB7CA1B51
:1018E000DB0B0FB6F894DEBF0FBECDBF09942A887C
:1018F000398848885F846E847D848C849B84AA8424
:10190000B984C884DF80EE80FD800C811B81AA81B0
:10191000B981CE0FD11D0FB6F894DEBF0FBECDBF7B
:10192000ED010895A1E21A2EAA1BBB1BFD010DC0FB
:10193000AA1FBB1FEE1FFF1FA217B307E407F5077F
:1019400020F0A21BB30BE40BF50B661F771F881F5B
:10195000991F1A9469F760957095809590959B01F1
:10196000AC01BD01CF010895EE0FFF1F0590F4916A
:10197000E02D0994DF93CF939F92A0E49A2E002448
:10198000D001E001F00116950795F794E794D794FC
:10199000C794B794A79448F41068A20FB31FC41F4C
:1019A000D51FE61FF71F081E191E220F331F441FE5
:1019B000551F661F771F881F991F9A9421F79D0155
:1019C000AE01BF01C00111249F90CF91DF91089516
:1019D000A0E0B0E0EDEEFCE074CFEC01688179812D
:1019E0008A819B81611571058105910521F464E26D
:1019F00079ED8BE597E02DE133EF41E050E022DF18
:101A000049015A0127EA31E440E050E037DF69013B
:101A10007A01C501B4012CEE34EF4FEF5FEF2EDFFA
:101A2000022F132F9A01D701C601800F911FA21F09
:101A3000B31FB7FF03C00197A109B04888839983FA
:101A4000AA83BB83BC01CD019F77CDB7DEB7ECE0A5
:101A500054CFBEDF089580E091E0BADF089560932F
:101A60000001709301018093020190930301089596
:101A7000E199FECF9FBB8EBBE09A99278DB3089565
:101A8000262FE199FECF1CBA9FBB8EBB2DBB0FB694
:101A9000F894E29AE19A0FBE01960895F894FFCF68
:101AA000010000000000803F0000803F0000803FF8
:101AB0005A00000070420180050000FFFF2D00B6B3
:041AC00000540300CB
:00000001FF
